:01800000007F
:09800B00758CDC758A0005083251
:20810000A5E5E0A5FDFF00000000000000000000000000000000000000000000FFFFFFFF58
:028120007200EB
:2081400075810F90F002E4F0438901D2AFD2A9D28C128157021954058105810581740078C6
:20816000FE1283CAF67400F508740075F0001818F608A6F078FC1283CAE60886F07B647C0C
:208180000012844E45F070030281F6801678FC1283CAE60886F012843418F608A6F0128401
:2081A0003D80D1E5081283F57B0A1283EC12844E45F070030281BA0281A37400F50874C917
:2081C00075F084C0E0C0F078FC1283CAE61283F5C0E0C0F0740275F0001282101581158128
:2081E00015811581E5906480F59078FE1283CAE604F61402818D74D975F084C0E0C0F01204
:2082000082211581158112824C1581158115812223F42581F812849F12825C12849F028238
:208220002B78FB1283CA8682088683E0602D12823AA380F778FB1283CAE63099FDC299F505
:2082400099B40A17740D80F2E430980C3098FDC298E599B40D02740A75F000221283A386E2
:208260008208868308E4FEFFE070061283A3E4F022B42551A3E0B42D05430780A3E0B4303A
:208280000343074024D0B40A00500BCE75F00AA42EFEA3E080EEE0B46413E60886F030F7B0
:2082A00008430720128444A6F018F68003B4750543070A8021B478054307108019B46F10D1
:2082C00043070880111283A3F0A31283A3A38095B462624307027A00C004C005C006C007AC
:2082E000AB0753031F7C00E60886F01283FEA6F018F6EDD007D006D005D0042430B43A00BB
:2083000040022407C0E00AE645F070CC1283A3A902EF30E505742DF0A30A1283ACD0E0F0E4
:20832000A3D9FA0808EF30E7A1EAC39E509C7420F0A30A80F4B4630DAA011283A31283ACEC
:20834000E6F0A380DEB47331C082C08386820886837A00E06004A30A80F986831886821231
:2083600083A31283AC1283A3E0A31283A36004F0A380F2D005D00480AAB4691B86017A002E
:20838000E76004090A80F91283A31283AC8601E76091F009A380F8F97A011283A31283AC2D
:2083A000E9809ECDC583CDCCC582CC22EE601A8FF020F715C002EAC39E500C742030F6029B
:2083C0007430F0A30A80EFD00222C82581C822C92581C97A0022D083D082CF2581F581CF6E
:2083E000C082C08322CF2581F581CF227C00CB30E7011CCB2275F00030E70215F022C0022B
:20840000C001AAF0F97E007D007F11C3E933F9EA33FADF08F5F0E9D001D00222ED33FDEE09
:2084200033FEC3ED9BF5F0EE9C40E0ADF0FED380DB12843404700205F02212843D14B4FF77
:208440000215F02212843DF4C5F0F4C5F0221284814029801E12848140227017801E12845A
:208460008140107017800C128481501080051284956009E4F5F02212849560F7E4F5F0044E
:2084800022C39BC5F09C20E70720D207C345F02220D2F9D322C5F0C39C7003E5F09B229061
:2084A000F002E0A360F8E0FFA3E0A3CF2582F582EF3583F58380EBFBE0CB22FCE0FBA3E051
:2084C000CC22FAE0F9A3E0CA2225752048656C6C6F20576F726C640A000A70726573732035
:0884E000616E79206B657900E3
:00000001FF
